:020000020000FC
:020000001FC01F
:02002C00F5C01D
:02003400F1C019
:10004000F89414E01EBF1FEF1DBF00241124139469
:10005000FF24FA942FE414E0F1E0E0E001921A9515
:10006000E9F7222433244424439455246624772436
:1000700088249924AA24A394BB24CC24DD24F4B896
:10008000F5B807B808B81CE01AB914E01BB900921B
:10009000C50013E31093C40016E01093C20018E1EA
:1000A0001093C1000092C00010916400177F10935C
:1000B000640010E0109389001AEF1093880012E09A
:1000C00010936F00009282000092800019E010935C
:1000D000810078944091C00047FFFCCF4091C6005A
:1000E0008DE00E942C018AE00E942C01842F0E9446
:1000F0002C01142F107F1039B9F44091C00047FF34
:10010000FCCF4091C600F2E0E0EA440FE40F08F4AF
:10011000F39565907590332422244091C00047FFE9
:10012000FCCF4091C600D6CF103879F466247724EE
:100130004091C00047FFFCCF4091C6004091C000F5
:1001400047FFFCCF4091C600C5CF413619F4289A2D
:100150000C946A004A3719F428980C946A004337C3
:1001600019F4299A0C946A00483719F429980C94C8
:100170006A00443619F42A9A0C946A00433619F43A
:100180002A980C946A00463619F42B9A0C946A004B
:10019000463719F42B980C946A00473619F42C9AB8
:1001A0000C946A00423619F42C980C946A00483674
:1001B00019F42D9A0C946A004E3619F42D980C946B
:1001C0006A00413370F04A3364F4F2E0E0EA440F2D
:1001D000E40F08F4F39565907590222433240C9471
:1001E0006A00493641F447FE80E347FC81E30E9400
:1001F0002C010C946A00443741F4319B80E331991F
:1002000081E30E942C010C946A00403321F466249F
:1002100077240C946A005ECF5FB7662019F47720CC
:1002200009F418C0261469F4371459F43EE1222465
:1002300033242C9B02C02C9801C02C9A2A982D980C
:1002400009C0239409F43394332321F03A9511F42F
:100250002A982D9A5FBF1895E090C000E5FEFCCF6C
:100260008093C6000895466C6F707079204D4944A4
:1002700049202D20436F707972696768742032308D
:100280003039202D204D69636861656C204B6F68A3
:100290006E202D2056657273696F6E20302E3035BA
:1002A000490F6E0E9E0DDB0C220C740BCF0A340A24
:1002B000A109170994081908A4073707CF066D0686
:1002C0001106BA0567051A05D0048B044A040C040C
:1002D000D2039B03670336030803DD02B3028D02DA
:1002E0006802450225020602E901CD01B3019B0126
:1002F00084016E01590146013401220112010301FA
:10030000F400E600D900CD00C200B700AC00A300A5
:100310009A009100890081007A0073006C006600E9
:1003200061005B00560051004D0048004400400051
:100330003D0039003600330030002D002B0028002E
:1003400026002400220020001E001C001B001900B3
:100350001800160015001400130012001100100000
:100360000F000E000D000C000C000B000A000A002C
:100370000900090008000800070007000600060041
:100380000600050005000500040004000400040048
:100390000300030003000300030002000200020048
:00000001FF
